 sunmscapi

 Timestamp is 6710e051 (Thu Oct 17 10:00:49 2024)

 Preferred load address is 10000000

 Start         Length     Name                   Class
 0001:00000000 00000020H .text$di                CODE
 0001:00000020 00003a77H .text$mn                CODE
 0001:00003a97 0000001dH .text$x                 CODE
 0002:00000000 00000170H .idata$5                DATA
 0002:00000170 00000008H .00cfg                  DATA
 0002:00000178 00000004H .CRT$XCA                DATA
 0002:0000017c 00000004H .CRT$XCU                DATA
 0002:00000180 00000004H .CRT$XCZ                DATA
 0002:00000184 00000004H .CRT$XIA                DATA
 0002:00000188 00000004H .CRT$XIZ                DATA
 0002:0000018c 00000004H .CRT$XPA                DATA
 0002:00000190 00000004H .CRT$XPZ                DATA
 0002:00000194 00000004H .CRT$XTA                DATA
 0002:00000198 00000008H .CRT$XTZ                DATA
 0002:0000019c 00000000H .gfids$y                DATA
 0002:000001a0 00000760H .rdata                  DATA
 0002:00000900 00000000H .rdata$CastGuardVftablesA DATA
 0002:00000900 00000000H .rdata$CastGuardVftablesC DATA
 0002:00000900 0000012cH .rdata$r                DATA
 0002:00000a2c 00000008H .rdata$sxdata           DATA
 0002:00000a34 00000064H .rdata$voltmd           DATA
 0002:00000a98 00000360H .rdata$zzzdbg           DATA
 0002:00000df8 00000004H .rtc$IAA                DATA
 0002:00000dfc 00000004H .rtc$IZZ                DATA
 0002:00000e00 00000004H .rtc$TAA                DATA
 0002:00000e04 00000004H .rtc$TZZ                DATA
 0002:00000e08 000003d8H .xdata$x                DATA
 0002:000011e0 0000060cH .edata                  DATA
 0002:000017ec 000000dcH .idata$2                DATA
 0002:000018c8 00000014H .idata$3                DATA
 0002:000018dc 00000170H .idata$4                DATA
 0002:00001a4c 000007daH .idata$6                DATA
 0003:00000000 00000014H .data                   DATA
 0003:00000014 00000060H .data$r                 DATA
 0003:00000074 0000001cH .data$rs                DATA
 0003:00000090 00000374H .bss                    DATA
 0004:00000000 00000060H .rsrc$01                DATA
 0004:00000060 00000320H .rsrc$02                DATA

  Address         Publics by Value              Rva+Base       Lib:Object

 0000:00000000       ___AbsoluteZero            00000000     <absolute>
 0000:00000000       ___arm64x_extra_rfe_table  00000000     <absolute>
 0000:00000000       ___arm64x_extra_rfe_table_size 00000000     <absolute>
 0000:00000000       ___arm64x_native_entrypoint 00000000     <absolute>
 0000:00000000       ___arm64x_redirection_metadata 00000000     <absolute>
 0000:00000000       ___arm64x_redirection_metadata_count 00000000     <absolute>
 0000:00000000       ___dynamic_value_reloc_table 00000000     <absolute>
 0000:00000000       ___enclave_config          00000000     <absolute>
 0000:00000000       ___guard_check_icall_a64n_fptr 00000000     <absolute>
 0000:00000000       ___guard_eh_cont_count     00000000     <absolute>
 0000:00000000       ___guard_eh_cont_table     00000000     <absolute>
 0000:00000000       ___guard_fids_count        00000000     <absolute>
 0000:00000000       ___guard_fids_table        00000000     <absolute>
 0000:00000000       ___guard_iat_count         00000000     <absolute>
 0000:00000000       ___guard_iat_table         00000000     <absolute>
 0000:00000000       ___guard_longjmp_count     00000000     <absolute>
 0000:00000000       ___guard_longjmp_table     00000000     <absolute>
 0000:00000000       ___hybrid_auxiliary_delayload_iat 00000000     <absolute>
 0000:00000000       ___hybrid_auxiliary_delayload_iat_copy 00000000     <absolute>
 0000:00000000       ___hybrid_auxiliary_iat    00000000     <absolute>
 0000:00000000       ___hybrid_auxiliary_iat_copy 00000000     <absolute>
 0000:00000000       ___hybrid_code_map         00000000     <absolute>
 0000:00000000       ___hybrid_code_map_count   00000000     <absolute>
 0000:00000000       ___hybrid_image_info_bitfield 00000000     <absolute>
 0000:00000000       ___x64_code_ranges_to_entry_points 00000000     <absolute>
 0000:00000000       ___x64_code_ranges_to_entry_points_count 00000000     <absolute>
 0000:00000002       ___safe_se_handler_count   00000002     <absolute>
 0000:00000100       ___guard_flags             00000100     <absolute>
 0000:00000000       ___ImageBase               10000000     <linker-defined>
 0001:00000020       ?CallStaticObjectMethod@JNIEnv_@@QAAPAV_jobject@@PAV_jclass@@PAU_jmethodID@@ZZ 10001020 f i security.obj
 0001:0000003b       ?CallVoidMethod@JNIEnv_@@QAAXPAV_jobject@@PAU_jmethodID@@ZZ 1000103b f i security.obj
 0001:00000056       ?NewObject@JNIEnv_@@QAAPAV_jobject@@PAV_jclass@@PAU_jmethodID@@ZZ 10001056 f i security.obj
 0001:0000006e       _GetCertificateChain       1000106e f   security.obj
 0001:000000b1       _Java_sun_security_mscapi_CKeyPairGenerator_00024RSA_generateCKeyPair@20 100010b1 f   security.obj
 0001:000001d0       _Java_sun_security_mscapi_CKeyStore_destroyKeyContainer@12 100011d0 f   security.obj
 0001:00000262       _Java_sun_security_mscapi_CKeyStore_generateRSAPrivateKeyBlob@44 10001262 f   security.obj
 0001:0000028f       _Java_sun_security_mscapi_CKeyStore_loadKeysOrCertificateChains@12 1000128f f   security.obj
 0001:000009be       _Java_sun_security_mscapi_CKeyStore_removeCertificate@24 100019be f   security.obj
 0001:00000b99       _Java_sun_security_mscapi_CKeyStore_storeCertificate@40 10001b99 f   security.obj
 0001:00000f70       _Java_sun_security_mscapi_CKeyStore_storePrivateKey@24 10001f70 f   security.obj
 0001:000010b6       _Java_sun_security_mscapi_CKey_cleanUp@24 100020b6 f   security.obj
 0001:000010f3       _Java_sun_security_mscapi_CKey_getContainerName@16 100020f3 f   security.obj
 0001:00001155       _Java_sun_security_mscapi_CKey_getKeyType@16 10002155 f   security.obj
 0001:000011e4       _Java_sun_security_mscapi_CPublicKey_00024CRSAPublicKey_getExponent@12 100021e4 f   security.obj
 0001:000012f0       _Java_sun_security_mscapi_CPublicKey_00024CRSAPublicKey_getModulus@12 100022f0 f   security.obj
 0001:00001424       _Java_sun_security_mscapi_CPublicKey_getPublicKeyBlob@24 10002424 f   security.obj
 0001:000015a4       _Java_sun_security_mscapi_CRSACipher_encryptDecrypt@32 100025a4 f   security.obj
 0001:00001756       _Java_sun_security_mscapi_CSignature_00024RSA_generatePublicKeyBlob@20 10002756 f   security.obj
 0001:00001779       _Java_sun_security_mscapi_CSignature_importECPublicKey@20 10002779 f   security.obj
 0001:000018a6       _Java_sun_security_mscapi_CSignature_importPublicKey@20 100028a6 f   security.obj
 0001:000019d4       _Java_sun_security_mscapi_CSignature_signCngHash@44 100029d4 f   security.obj
 0001:00001c02       _Java_sun_security_mscapi_CSignature_signHash@40 10002c02 f   security.obj
 0001:00001e6d       _Java_sun_security_mscapi_CSignature_verifyCngSignedHash@52 10002e6d f   security.obj
 0001:00002047       _Java_sun_security_mscapi_CSignature_verifySignedHash@44 10003047 f   security.obj
 0001:00002269       _Java_sun_security_mscapi_PRNG_generateSeed@16 10003269 f   security.obj
 0001:000023cf       _MapHashAlgorithm          100033cf f   security.obj
 0001:000024d8       _MapHashIdentifier         100034d8 f   security.obj
 0001:0000258d       _ThrowException            1000358d f   security.obj
 0001:00002603       _ThrowExceptionWithMessage 10003603 f   security.obj
 0001:00002623       ___local_stdio_printf_options 10003623 f i security.obj
 0001:00002629       __vfprintf_l               10003629 f i security.obj
 0001:0000264d       __vsnprintf_l              1000364d f i security.obj
 0001:00002680       _convertToLittleEndian     10003680 f   security.obj
 0001:0000275e       _dump                      1000375e f   security.obj
 0001:00002859       _fprintf                   10003859 f i security.obj
 0001:00002871       _generateKeyBlob           10003871 f   security.obj
 0001:00002a88       _new[]                     10003a88 f   security.obj
 0001:00002ab9       _printf                    10003ab9 f i security.obj
 0001:00002ad7       _sprintf                   10003ad7 f i security.obj
 0001:00002af1       _NCryptOpenStorageProvider@12 10003af1 f   ncrypt:ncrypt.dll
 0001:00002af7       _NCryptGetProperty@24      10003af7 f   ncrypt:ncrypt.dll
 0001:00002afd       _NCryptImportKey@32        10003afd f   ncrypt:ncrypt.dll
 0001:00002b03       _NCryptExportKey@32        10003b03 f   ncrypt:ncrypt.dll
 0001:00002b09       _NCryptSignHash@32         10003b09 f   ncrypt:ncrypt.dll
 0001:00002b0f       _NCryptVerifySignature@28  10003b0f f   ncrypt:ncrypt.dll
 0001:00002b15       _NCryptFreeObject@4        10003b15 f   ncrypt:ncrypt.dll
 0001:00002b1b       _NCryptTranslateHandle@24  10003b1b f   ncrypt:ncrypt.dll
 0001:00002b21       ??_V@YAXPAX@Z              10003b21 f   MSVCRT:delete_array.obj
 0001:00002b26       ??_U@YAPAXIABUnothrow_t@std@@@Z 10003b26 f   MSVCRT:new_array_nothrow.obj
 0001:00002b2f       @__security_check_cookie@4 10003b2f f   MSVCRT:secchk.obj
 0001:00002b40       __SEH_prolog4              10003b40 f   MSVCRT:sehprolg4.obj
 0001:00002b90       __SEH_prolog4_GS           10003b90 f   MSVCRT:sehprolg4gs.obj
 0001:00002be0       __except_handler4          10003be0 f   MSVCRT:chandler4gs.obj
 0001:00002f4f       __DllMainCRTStartup@12     10003f4f f   MSVCRT:dll_dllmain.obj
 0001:00002f72       ??3@YAXPAX@Z               10003f72 f   MSVCRT:delete_scalar.obj
 0001:00002f77       ??2@YAPAXIABUnothrow_t@std@@@Z 10003f77 f   MSVCRT:new_scalar_nothrow.obj
 0001:00002fcc       ___raise_securityfailure   10003fcc f   MSVCRT:gs_report.obj
 0001:00002ff4       ___report_gsfailure        10003ff4 f   MSVCRT:gs_report.obj
 0001:0000313b       ___security_init_cookie    1000413b f   MSVCRT:gs_support.obj
 0001:00003186       _DllMain@12                10004186 f   MSVCRT:dll_dllmain_stub.obj
 0001:000031a8       ?__scrt_initialize_type_info@@YAXXZ 100041a8 f   MSVCRT:tncleanup.obj
 0001:000031b4       ?__scrt_uninitialize_type_info@@YAXXZ 100041b4 f   MSVCRT:tncleanup.obj
 0001:000031c0       ___local_stdio_scanf_options 100041c0 f i MSVCRT:default_local_stdio_options.obj
 0001:000031c6       ___scrt_initialize_default_local_stdio_options 100041c6 f   MSVCRT:default_local_stdio_options.obj
 0001:00003227       ___scrt_acquire_startup_lock 10004227 f   MSVCRT:utility.obj
 0001:00003259       ___scrt_dllmain_after_initialize_c 10004259 f   MSVCRT:utility.obj
 0001:00003284       ___scrt_dllmain_before_initialize_c 10004284 f   MSVCRT:utility.obj
 0001:00003292       ___scrt_dllmain_crt_thread_attach 10004292 f   MSVCRT:utility.obj
 0001:000032b1       ___scrt_dllmain_crt_thread_detach 100042b1 f   MSVCRT:utility.obj
 0001:000032be       ___scrt_dllmain_exception_filter 100042be f   MSVCRT:utility.obj
 0001:000032f2       ___scrt_dllmain_uninitialize_c 100042f2 f   MSVCRT:utility.obj
 0001:00003315       ___scrt_dllmain_uninitialize_critical 10004315 f   MSVCRT:utility.obj
 0001:00003322       ___scrt_initialize_crt     10004322 f   MSVCRT:utility.obj
 0001:0000335b       ___scrt_initialize_onexit_tables 1000435b f   MSVCRT:utility.obj
 0001:000033e2       ___scrt_is_nonwritable_in_current_image 100043e2 f   MSVCRT:utility.obj
 0001:00003476       ___scrt_release_startup_lock 10004476 f   MSVCRT:utility.obj
 0001:00003493       ___scrt_uninitialize_crt   10004493 f   MSVCRT:utility.obj
 0001:000034bb       ___scrt_get_dyn_tls_init_callback 100044bb f   MSVCRT:dyn_tls_init.obj
 0001:000034c1       ___scrt_fastfail           100044c1 f   MSVCRT:utility_desktop.obj
 0001:000035dc       __crt_debugger_hook        100045dc f   MSVCRT:utility_desktop.obj
 0001:000035e4       __RTC_Initialize           100045e4 f   MSVCRT:initsect.obj
 0001:00003610       __RTC_Terminate            10004610 f   MSVCRT:initsect.obj
 0001:0000363c       @_guard_check_icall_nop@4  1000463c f i MSVCRT:guard_support.obj
 0001:0000363f       ??2@YAPAXI@Z               1000463f f   MSVCRT:new_scalar.obj
 0001:0000366f       ___isa_available_init      1000466f f   MSVCRT:cpu_disp.obj
 0001:00003843       __get_startup_argv_mode    10004843 f   MSVCRT:argv_mode.obj
 0001:00003847       ___scrt_is_ucrt_dll_in_use 10004847 f   MSVCRT:ucrt_detection.obj
 0001:00003853       ??0bad_alloc@std@@QAE@ABV01@@Z 10004853 f i MSVCRT:throw_bad_alloc.obj
 0001:0000386e       ??0bad_alloc@std@@QAE@XZ   1000486e f i MSVCRT:throw_bad_alloc.obj
 0001:00003886       ??0bad_array_new_length@std@@QAE@ABV01@@Z 10004886 f i MSVCRT:throw_bad_alloc.obj
 0001:000038a1       ??0bad_array_new_length@std@@QAE@XZ 100048a1 f i MSVCRT:throw_bad_alloc.obj
 0001:000038b9       ??0exception@std@@QAE@ABV01@@Z 100048b9 f i MSVCRT:throw_bad_alloc.obj
 0001:000038e5       ??1bad_alloc@std@@UAE@XZ   100048e5 f i MSVCRT:throw_bad_alloc.obj
 0001:000038e5       ??1bad_array_new_length@std@@UAE@XZ 100048e5 f i MSVCRT:throw_bad_alloc.obj
 0001:000038f6       ??_Ebad_alloc@std@@UAEPAXI@Z 100048f6 f i MSVCRT:throw_bad_alloc.obj
 0001:000038f6       ??_Ebad_array_new_length@std@@UAEPAXI@Z 100048f6 f i MSVCRT:throw_bad_alloc.obj
 0001:000038f6       ??_Eexception@std@@UAEPAXI@Z 100048f6 f i MSVCRT:throw_bad_alloc.obj
 0001:000038f6       ??_Gbad_alloc@std@@UAEPAXI@Z 100048f6 f i MSVCRT:throw_bad_alloc.obj
 0001:000038f6       ??_Gbad_array_new_length@std@@UAEPAXI@Z 100048f6 f i MSVCRT:throw_bad_alloc.obj
 0001:000038f6       ??_Gexception@std@@UAEPAXI@Z 100048f6 f i MSVCRT:throw_bad_alloc.obj
 0001:00003923       ?__scrt_throw_std_bad_alloc@@YAXXZ 10004923 f   MSVCRT:throw_bad_alloc.obj
 0001:00003940       ?__scrt_throw_std_bad_array_new_length@@YAXXZ 10004940 f   MSVCRT:throw_bad_alloc.obj
 0001:0000395d       ?what@exception@std@@UBEPBDXZ 1000495d f i MSVCRT:throw_bad_alloc.obj
 0001:0000396a       ??3@YAXPAXI@Z              1000496a f   MSVCRT:delete_scalar_size.obj
 0001:00003978       ??_Etype_info@@UAEPAXI@Z   10004978 f i MSVCRT:std_type_info_static.obj
 0001:00003978       ??_Gtype_info@@UAEPAXI@Z   10004978 f i MSVCRT:std_type_info_static.obj
 0001:0000399b       _memcpy                    1000499b f   vcruntime:VCRUNTIME140.dll
 0001:000039a1       _memset                    100049a1 f   vcruntime:VCRUNTIME140.dll
 0001:000039a7       __except_handler4_common   100049a7 f   vcruntime:VCRUNTIME140.dll
 0001:000039ad       ___CxxFrameHandler3        100049ad f   vcruntime:VCRUNTIME140.dll
 0001:000039b3       ___std_type_info_destroy_list 100049b3 f   vcruntime:VCRUNTIME140.dll
 0001:000039b9       ___std_exception_copy      100049b9 f   vcruntime:VCRUNTIME140.dll
 0001:000039bf       ___std_exception_destroy   100049bf f   vcruntime:VCRUNTIME140.dll
 0001:000039c5       __CxxThrowException@8      100049c5 f   vcruntime:VCRUNTIME140.dll
 0001:000039cb       _strcmp                    100049cb f   ucrt:api-ms-win-crt-string-l1-1-0.dll
 0001:000039d1       _strcpy                    100049d1 f   ucrt:api-ms-win-crt-string-l1-1-0.dll
 0001:000039d7       __initterm                 100049d7 f   ucrt:api-ms-win-crt-runtime-l1-1-0.dll
 0001:000039dd       __initterm_e               100049dd f   ucrt:api-ms-win-crt-runtime-l1-1-0.dll
 0001:000039e3       _free                      100049e3 f   ucrt:api-ms-win-crt-heap-l1-1-0.dll
 0001:000039e9       __seh_filter_dll           100049e9 f   ucrt:api-ms-win-crt-runtime-l1-1-0.dll
 0001:000039ef       __configure_narrow_argv    100049ef f   ucrt:api-ms-win-crt-runtime-l1-1-0.dll
 0001:000039f5       __initialize_narrow_environment 100049f5 f   ucrt:api-ms-win-crt-runtime-l1-1-0.dll
 0001:000039fb       __initialize_onexit_table  100049fb f   ucrt:api-ms-win-crt-runtime-l1-1-0.dll
 0001:00003a01       __execute_onexit_table     10004a01 f   ucrt:api-ms-win-crt-runtime-l1-1-0.dll
 0001:00003a07       __cexit                    10004a07 f   ucrt:api-ms-win-crt-runtime-l1-1-0.dll
 0001:00003a0d       __callnewh                 10004a0d f   ucrt:api-ms-win-crt-heap-l1-1-0.dll
 0001:00003a13       _malloc                    10004a13 f   ucrt:api-ms-win-crt-heap-l1-1-0.dll
 0001:00003a19       __filter_x86_sse2_floating_point_exception 10004a19 f   MSVCRT:x86_exception_filter.obj
 0001:00003a19       __filter_x86_sse2_floating_point_exception_default 10004a19 f   MSVCRT:x86_exception_filter.obj
 0001:00003a91       ___acrt_initialize         10004a91 f   MSVCRT:ucrt_stubs.obj
 0001:00003a91       ___acrt_thread_attach      10004a91 f   MSVCRT:ucrt_stubs.obj
 0001:00003a91       ___acrt_thread_detach      10004a91 f   MSVCRT:ucrt_stubs.obj
 0001:00003a91       ___acrt_uninitialize       10004a91 f   MSVCRT:ucrt_stubs.obj
 0001:00003a91       ___acrt_uninitialize_critical 10004a91 f   MSVCRT:ucrt_stubs.obj
 0001:00003a91       ___scrt_stub_for_acrt_initialize 10004a91 f   MSVCRT:ucrt_stubs.obj
 0001:00003a91       ___scrt_stub_for_acrt_thread_attach 10004a91 f   MSVCRT:ucrt_stubs.obj
 0001:00003a91       ___scrt_stub_for_acrt_thread_detach 10004a91 f   MSVCRT:ucrt_stubs.obj
 0001:00003a91       ___scrt_stub_for_acrt_uninitialize 10004a91 f   MSVCRT:ucrt_stubs.obj
 0001:00003a91       ___scrt_stub_for_acrt_uninitialize_critical 10004a91 f   MSVCRT:ucrt_stubs.obj
 0001:00003a91       ___vcrt_initialize         10004a91 f   MSVCRT:ucrt_stubs.obj
 0001:00003a91       ___vcrt_thread_attach      10004a91 f   MSVCRT:ucrt_stubs.obj
 0001:00003a91       ___vcrt_thread_detach      10004a91 f   MSVCRT:ucrt_stubs.obj
 0001:00003a91       ___vcrt_uninitialize       10004a91 f   MSVCRT:ucrt_stubs.obj
 0001:00003a91       ___vcrt_uninitialize_critical 10004a91 f   MSVCRT:ucrt_stubs.obj
 0001:00003a94       ___scrt_stub_for_is_c_termination_complete 10004a94 f   MSVCRT:ucrt_stubs.obj
 0001:00003a94       __is_c_termination_complete 10004a94 f   MSVCRT:ucrt_stubs.obj
 0002:00000000       __imp__CryptGenKey@16      10005000     advapi32:ADVAPI32.dll
 0002:00000004       __imp__CryptVerifySignatureA@24 10005004     advapi32:ADVAPI32.dll
 0002:00000008       __imp__CryptSignHashA@24   10005008     advapi32:ADVAPI32.dll
 0002:0000000c       __imp__CryptDestroyHash@4  1000500c     advapi32:ADVAPI32.dll
 0002:00000010       __imp__CryptCreateHash@20  10005010     advapi32:ADVAPI32.dll
 0002:00000014       __imp__CryptDecrypt@24     10005014     advapi32:ADVAPI32.dll
 0002:00000018       __imp__CryptEncrypt@28     10005018     advapi32:ADVAPI32.dll
 0002:0000001c       __imp__CryptImportKey@24   1000501c     advapi32:ADVAPI32.dll
 0002:00000020       __imp__CryptExportKey@24   10005020     advapi32:ADVAPI32.dll
 0002:00000024       __imp__CryptGetUserKey@12  10005024     advapi32:ADVAPI32.dll
 0002:00000028       __imp__CryptGenRandom@12   10005028     advapi32:ADVAPI32.dll
 0002:0000002c       __imp__CryptGetProvParam@20 1000502c     advapi32:ADVAPI32.dll
 0002:00000030       __imp__CryptSetHashParam@16 10005030     advapi32:ADVAPI32.dll
 0002:00000034       __imp__CryptGetKeyParam@20 10005034     advapi32:ADVAPI32.dll
 0002:00000038       __imp__CryptSetKeyParam@16 10005038     advapi32:ADVAPI32.dll
 0002:0000003c       __imp__CryptAcquireContextA@20 1000503c     advapi32:ADVAPI32.dll
 0002:00000040       __imp__CryptReleaseContext@8 10005040     advapi32:ADVAPI32.dll
 0002:00000044       __imp__CryptDestroyKey@4   10005044     advapi32:ADVAPI32.dll
 0002:00000048       \177ADVAPI32_NULL_THUNK_DATA 10005048     advapi32:ADVAPI32.dll
 0002:0000004c       __imp__CertDeleteCertificateFromStore@4 1000504c     Crypt32:CRYPT32.dll
 0002:00000050       __imp__CertFreeCertificateChain@4 10005050     Crypt32:CRYPT32.dll
 0002:00000054       __imp__CertGetCertificateChain@32 10005054     Crypt32:CRYPT32.dll
 0002:00000058       __imp__CertOpenSystemStoreA@8 10005058     Crypt32:CRYPT32.dll
 0002:0000005c       __imp__CertGetNameStringA@24 1000505c     Crypt32:CRYPT32.dll
 0002:00000060       __imp__CryptAcquireCertificatePrivateKey@24 10005060     Crypt32:CRYPT32.dll
 0002:00000064       __imp__CertGetPublicKeyLength@8 10005064     Crypt32:CRYPT32.dll
 0002:00000068       __imp__CertCloseStore@8    10005068     Crypt32:CRYPT32.dll
 0002:0000006c       __imp__CertAddCertificateContextToStore@16 1000506c     Crypt32:CRYPT32.dll
 0002:00000070       __imp__CertSetCertificateContextProperty@16 10005070     Crypt32:CRYPT32.dll
 0002:00000074       __imp__CertFreeCertificateContext@4 10005074     Crypt32:CRYPT32.dll
 0002:00000078       __imp__CertCreateCertificateContext@12 10005078     Crypt32:CRYPT32.dll
 0002:0000007c       __imp__CertFindCertificateInStore@24 1000507c     Crypt32:CRYPT32.dll
 0002:00000080       __imp__CertEnumCertificatesInStore@8 10005080     Crypt32:CRYPT32.dll
 0002:00000084       \177CRYPT32_NULL_THUNK_DATA 10005084     Crypt32:CRYPT32.dll
 0002:00000088       __imp__IsDebuggerPresent@0 10005088     kernel32:KERNEL32.dll
 0002:0000008c       __imp__InitializeSListHead@4 1000508c     kernel32:KERNEL32.dll
 0002:00000090       __imp__DisableThreadLibraryCalls@4 10005090     kernel32:KERNEL32.dll
 0002:00000094       __imp__GetSystemTimeAsFileTime@4 10005094     kernel32:KERNEL32.dll
 0002:00000098       __imp__GetCurrentThreadId@0 10005098     kernel32:KERNEL32.dll
 0002:0000009c       __imp__GetCurrentProcessId@0 1000509c     kernel32:KERNEL32.dll
 0002:000000a0       __imp__QueryPerformanceCounter@4 100050a0     kernel32:KERNEL32.dll
 0002:000000a4       __imp__GetLastError@0      100050a4     kernel32:KERNEL32.dll
 0002:000000a8       __imp__FormatMessageA@28   100050a8     kernel32:KERNEL32.dll
 0002:000000ac       __imp__UnhandledExceptionFilter@4 100050ac     kernel32:KERNEL32.dll
 0002:000000b0       __imp__SetUnhandledExceptionFilter@4 100050b0     kernel32:KERNEL32.dll
 0002:000000b4       __imp__GetCurrentProcess@0 100050b4     kernel32:KERNEL32.dll
 0002:000000b8       __imp__TerminateProcess@8  100050b8     kernel32:KERNEL32.dll
 0002:000000bc       __imp__IsProcessorFeaturePresent@4 100050bc     kernel32:KERNEL32.dll
 0002:000000c0       \177KERNEL32_NULL_THUNK_DATA 100050c0     kernel32:KERNEL32.dll
 0002:000000c4       __imp____std_exception_destroy 100050c4     vcruntime:VCRUNTIME140.dll
 0002:000000c8       __imp____std_exception_copy 100050c8     vcruntime:VCRUNTIME140.dll
 0002:000000cc       __imp____std_type_info_destroy_list 100050cc     vcruntime:VCRUNTIME140.dll
 0002:000000d0       __imp____CxxFrameHandler3  100050d0     vcruntime:VCRUNTIME140.dll
 0002:000000d4       __imp___except_handler4_common 100050d4     vcruntime:VCRUNTIME140.dll
 0002:000000d8       __imp__memset              100050d8     vcruntime:VCRUNTIME140.dll
 0002:000000dc       __imp__memcpy              100050dc     vcruntime:VCRUNTIME140.dll
 0002:000000e0       __imp___CxxThrowException@8 100050e0     vcruntime:VCRUNTIME140.dll
 0002:000000e4       \177VCRUNTIME140_NULL_THUNK_DATA 100050e4     vcruntime:VCRUNTIME140.dll
 0002:000000e8       __imp__mbstowcs            100050e8     ucrt:api-ms-win-crt-convert-l1-1-0.dll
 0002:000000ec       \177api-ms-win-crt-convert-l1-1-0_NULL_THUNK_DATA 100050ec     ucrt:api-ms-win-crt-convert-l1-1-0.dll
 0002:000000f0       __imp__getenv              100050f0     ucrt:api-ms-win-crt-environment-l1-1-0.dll
 0002:000000f4       \177api-ms-win-crt-environment-l1-1-0_NULL_THUNK_DATA 100050f4     ucrt:api-ms-win-crt-environment-l1-1-0.dll
 0002:000000f8       __imp__malloc              100050f8     ucrt:api-ms-win-crt-heap-l1-1-0.dll
 0002:000000fc       __imp___callnewh           100050fc     ucrt:api-ms-win-crt-heap-l1-1-0.dll
 0002:00000100       __imp__free                10005100     ucrt:api-ms-win-crt-heap-l1-1-0.dll
 0002:00000104       \177api-ms-win-crt-heap-l1-1-0_NULL_THUNK_DATA 10005104     ucrt:api-ms-win-crt-heap-l1-1-0.dll
 0002:00000108       __imp___initialize_onexit_table 10005108     ucrt:api-ms-win-crt-runtime-l1-1-0.dll
 0002:0000010c       __imp___cexit              1000510c     ucrt:api-ms-win-crt-runtime-l1-1-0.dll
 0002:00000110       __imp___execute_onexit_table 10005110     ucrt:api-ms-win-crt-runtime-l1-1-0.dll
 0002:00000114       __imp___initialize_narrow_environment 10005114     ucrt:api-ms-win-crt-runtime-l1-1-0.dll
 0002:00000118       __imp___configure_narrow_argv 10005118     ucrt:api-ms-win-crt-runtime-l1-1-0.dll
 0002:0000011c       __imp___initterm           1000511c     ucrt:api-ms-win-crt-runtime-l1-1-0.dll
 0002:00000120       __imp___initterm_e         10005120     ucrt:api-ms-win-crt-runtime-l1-1-0.dll
 0002:00000124       __imp___seh_filter_dll     10005124     ucrt:api-ms-win-crt-runtime-l1-1-0.dll
 0002:00000128       \177api-ms-win-crt-runtime-l1-1-0_NULL_THUNK_DATA 10005128     ucrt:api-ms-win-crt-runtime-l1-1-0.dll
 0002:0000012c       __imp____acrt_iob_func     1000512c     ucrt:api-ms-win-crt-stdio-l1-1-0.dll
 0002:00000130       __imp__fflush              10005130     ucrt:api-ms-win-crt-stdio-l1-1-0.dll
 0002:00000134       __imp____stdio_common_vfprintf 10005134     ucrt:api-ms-win-crt-stdio-l1-1-0.dll
 0002:00000138       __imp____stdio_common_vsprintf 10005138     ucrt:api-ms-win-crt-stdio-l1-1-0.dll
 0002:0000013c       \177api-ms-win-crt-stdio-l1-1-0_NULL_THUNK_DATA 1000513c     ucrt:api-ms-win-crt-stdio-l1-1-0.dll
 0002:00000140       __imp__strcpy              10005140     ucrt:api-ms-win-crt-string-l1-1-0.dll
 0002:00000144       __imp__strcmp              10005144     ucrt:api-ms-win-crt-string-l1-1-0.dll
 0002:00000148       \177api-ms-win-crt-string-l1-1-0_NULL_THUNK_DATA 10005148     ucrt:api-ms-win-crt-string-l1-1-0.dll
 0002:0000014c       __imp__NCryptSignHash@32   1000514c     ncrypt:ncrypt.dll
 0002:00000150       __imp__NCryptVerifySignature@28 10005150     ncrypt:ncrypt.dll
 0002:00000154       __imp__NCryptOpenStorageProvider@12 10005154     ncrypt:ncrypt.dll
 0002:00000158       __imp__NCryptImportKey@32  10005158     ncrypt:ncrypt.dll
 0002:0000015c       __imp__NCryptFreeObject@4  1000515c     ncrypt:ncrypt.dll
 0002:00000160       __imp__NCryptTranslateHandle@24 10005160     ncrypt:ncrypt.dll
 0002:00000164       __imp__NCryptGetProperty@24 10005164     ncrypt:ncrypt.dll
 0002:00000168       __imp__NCryptExportKey@32  10005168     ncrypt:ncrypt.dll
 0002:0000016c       \177ncrypt_NULL_THUNK_DATA 1000516c     ncrypt:ncrypt.dll
 0002:00000170       ___guard_check_icall_fptr  10005170     MSVCRT:guard_support.obj
 0002:00000174       ___castguard_check_failure_os_handled_fptr 10005174     MSVCRT:guard_support.obj
 0002:00000178       ___xc_a                    10005178     MSVCRT:initializers.obj
 0002:00000180       ___xc_z                    10005180     MSVCRT:initializers.obj
 0002:00000184       ___xi_a                    10005184     MSVCRT:initializers.obj
 0002:00000188       ___xi_z                    10005188     MSVCRT:initializers.obj
 0002:0000018c       ___xp_a                    1000518c     MSVCRT:initializers.obj
 0002:00000190       ___xp_z                    10005190     MSVCRT:initializers.obj
 0002:00000194       ___xt_a                    10005194     MSVCRT:initializers.obj
 0002:00000198       ___xt_z                    10005198     MSVCRT:initializers.obj
 0002:000001a0       ??_C@_0L@DCABDNEG@CAPI_TRACE@ 100051a0     security.obj
 0002:000001ac       ??_C@_0O@EEFELDNF@?$DN?$DN?$DN?$DN?5?$CFs?5?$DN?$DN?$DN?$DN?6@ 100051ac     security.obj
 0002:000001bc       ??_C@_06LNDOODMG@?$CF04x?3?5@ 100051bc     security.obj
 0002:000001c4       ??_C@_02KNHHEEKP@?5?5@     100051c4     security.obj
 0002:000001c8       ??_C@_05BFHEBJNP@?$CF02X?5@ 100051c8     security.obj
 0002:000001d0       ??_C@_03NDEAONJP@?5?5?5@   100051d0     security.obj
 0002:000001d4       ??_C@_01LFCBOECM@?4@       100051d4     security.obj
 0002:000001d8       ??_C@_02HAOIJKIC@?$CFc@    100051d8     security.obj
 0002:000001dc       ??_C@_01EEMJAFIK@?6@       100051dc     security.obj
 0002:000001e0       ??_C@_0O@NIPGCINC@Unknown?5error@ 100051e0     security.obj
 0002:000001f0       ??_C@_0CA@OCDEIOEB@Native?5memory?5allocation?5failed@ 100051f0     security.obj
 0002:00000210       ??_C@_0BL@ENCPOIKC@java?1lang?1OutOfMemoryError@ 10005210     security.obj
 0002:0000022c       ??_C@_03JAOICCJD@SHA@      1000522c     security.obj
 0002:00000230       ??_C@_04KPMLCNGO@SHA1@     10005230     security.obj
 0002:00000238       ??_C@_05HJMENKNE@SHA?91@   10005238     security.obj
 0002:00000240       ??_C@_08IPMGJMCA@SHA1?$CLMD5@ 10005240     security.obj
 0002:0000024c       ??_C@_07DKFLFLPF@SHA?9256@ 1000524c     security.obj
 0002:00000254       ??_C@_07LIAJMNEB@SHA?9384@ 10005254     security.obj
 0002:0000025c       ??_C@_07MEOJAOJE@SHA?9512@ 1000525c     security.obj
 0002:00000264       ??_C@_03GCGHEHKJ@MD5@      10005264     security.obj
 0002:00000268       ??_C@_03CNCGNBGO@MD2@      10005268     security.obj
 0002:0000026c       ??_C@_19DILNDFJH@?$AAS?$AAH?$AAA?$AA1@ 1000526c     security.obj
 0002:00000278       ??_C@_1O@HECGKAIN@?$AAS?$AAH?$AAA?$AA2?$AA5?$AA6@ 10005278     security.obj
 0002:00000288       ??_C@_1O@KOBLHLEG@?$AAS?$AAH?$AAA?$AA3?$AA8?$AA4@ 10005288     security.obj
 0002:00000298       ??_C@_1O@GKBAHMNF@?$AAS?$AAH?$AAA?$AA5?$AA1?$AA2@ 10005298     security.obj
 0002:000002a8       ??_C@_0CA@ODKEJAIA@java?1security?1ProviderException@ 100052a8     security.obj
 0002:000002c8       ??_C@_0CA@MACLKLAA@java?1security?1KeyStoreException@ 100052c8     security.obj
 0002:000002e8       ??_C@_0BE@GPOIDJOH@java?1util?1ArrayList@ 100052e8     security.obj
 0002:000002fc       ??_C@_03GAEACAIP@?$CI?$CJV@ 100052fc     security.obj
 0002:00000300       ??_C@_06FALKBLGB@?$DMinit?$DO@ 10005300     security.obj
 0002:00000308       ??_C@_0BM@MIKFLICJ@?$CI?$FLBLjava?1util?1Collection?$DL?$CJV@ 10005308     security.obj
 0002:00000324       ??_C@_0BE@HGBDNPAN@generateCertificate@ 10005324     security.obj
 0002:00000338       ??_C@_0CM@JPBKDHED@?$CILjava?1lang?1String?$DLLjava?1util?1C@ 10005338     security.obj
 0002:00000364       ??_C@_0BJ@POMOMMIJ@generateCertificateChain@ 10005364     security.obj
 0002:00000380       ??_C@_0DA@FHNPPNIC@?$CIZLjava?1lang?1String?$DLJJILjava?1ut@ 10005380     security.obj
 0002:000003b0       ??_C@_0BP@KJIOGBOH@generateKeyAndCertificateChain@ 100053b0     security.obj
 0002:000003d0       ??_C@_0P@LDACLLBM@MSCAPI?5?$CI?$CFld?$CJ?3?5@ 100053d0     security.obj
 0002:000003e0       ??_C@_0BL@JMBEPNBE@?9?9?9?9?9?9?9?9?9?9?9?9?9?9?9?9?9?9?9?9?9?9?9?9?9?9@ 100053e0     security.obj
 0002:000003fc       ??_C@_0BJ@LOMAEPIP@bHasNoPrivateKey?5?$DN?5TRUE?$CB@ 100053fc     security.obj
 0002:00000418       ??_C@_0BK@PBCGELBN@bHasNoPrivateKey?5?$DN?5TRUE?$CB?$CB@ 10005418     security.obj
 0002:00000434       ??_C@_09GGHMOLPI@CNG?5?$CFI64d@ 10005434     security.obj
 0002:00000440       ??_C@_0BB@DPFIGFPO@CAPI?5?$CFI64d?5?$CFI64d@ 10005440     security.obj
 0002:00000454       ??_C@_0M@MNGGKKAH@2?45?429?437?40@ 10005454     security.obj
 0002:00000460       ??_C@_06DJHOIPC@?$CFs?3?5?$CFs@ 10005460     security.obj
 0002:00000468       ??_C@_1BO@LONLFJGG@?$AAA?$AAl?$AAg?$AAo?$AAr?$AAi?$AAt?$AAh?$AAm?$AA?5?$AAN?$AAa?$AAm?$AAe@ 10005468     security.obj
 0002:00000488       ??_C@_0CC@FLCGHJKD@Unknown?5NCRYPT_ALGORITHM_PROPER@ 10005488     security.obj
 0002:000004ac       ??_C@_0BO@PMPHIPKH@GetCertificateChain?5failed?5?$CFd@ 100054ac     security.obj
 0002:000004cc       ??_C@_0CB@OJNKLEOL@java?1security?1SignatureExceptio@ 100054cc     security.obj
 0002:000004f0       ??_C@_0BM@BFBFCGA@Unrecognised?5hash?5algorithm@ 100054f0     security.obj
 0002:0000050c       ??_C@_1BM@HFKJNGID@?$AAE?$AAC?$AAC?$AAP?$AAU?$AAB?$AAL?$AAI?$AAC?$AAB?$AAL?$AAO?$AAB@ 1000550c     security.obj
 0002:00000528       ??_C@_0BL@LLOKBKPE@java?1security?1KeyException@ 10005528     security.obj
 0002:00000544       ??_C@_0BN@LEDKEDGO@sun?1security?1mscapi?1CKeyPair@ 10005544     security.obj
 0002:00000564       ??_C@_0BJ@HAHEHOOK@?$CILjava?1lang?1String?$DLJJI?$CJV@ 10005564     security.obj
 0002:00000580       ??_C@_09GDNFOKKF@Signature@ 10005580     security.obj
 0002:0000058c       ??_C@_08IGAGGAPJ@Exchange@ 1000558c     security.obj
 0002:00000598       ??_C@_03FKNCMABI@?$CFlu@   10005598     security.obj
 0002:0000059c       ??_C@_09MGFHLAFE@?$DMUnknown?$DO@ 1000559c     security.obj
 0002:000005a8       ??_C@_0CP@KCIKFHJG@java?1security?1cert?1CertificateP@ 100055a8     security.obj
 0002:000005d8       ??_C@_0N@GEJMMFOA@Invalid?5BLOB@ 100055d8     security.obj
 0002:000005e8       ??_C@_0BD@GEIFFJNC@Invalid?5key?5length@ 100055e8     security.obj
 0002:000005fc       ??_C@_0CC@LJIPPJAJ@java?1security?1InvalidKeyExcepti@ 100055fc     security.obj
 0002:00000620       ??_C@_0CA@BFBBJNML@sun?1security?1mscapi?1CPrivateKey@ 10005620     security.obj
 0002:00000640       ??_C@_0DJ@LBOEDAIF@?$CILjava?1lang?1String?$DLJJI?$CJLsun?1sec@ 10005640     security.obj
 0002:0000067c       ??_C@_02HAJCGGNB@of@       1000567c     security.obj
 0002:00000680       ??_C@_0BA@DCIOBNHG@NCryptImportKey@ 10005680     security.obj
 0002:00000690       ??_C@_1FA@OAAKELHB@?$AAM?$AAi?$AAc?$AAr?$AAo?$AAs?$AAo?$AAf?$AAt?$AA?5?$AAS?$AAo?$AAf?$AAt?$AAw@ 10005690     security.obj
 0002:000006e0       ??_C@_0BP@LCBGNOJP@sun?1security?1mscapi?1CPublicKey@ 100056e0     security.obj
 0002:00000700       ??_C@_0DI@BHHDKCOH@?$CILjava?1lang?1String?$DLJJI?$CJLsun?1sec@ 10005700     security.obj
 0002:00000738       ?nothrow@std@@3Unothrow_t@1@B 10005738     msvcprt:nothrow.obj
 0002:0000073c       __pDefaultRawDllMain       1000573c     MSVCRT:dll_dllmain.obj
 0002:0000073c       __pRawDllMain              1000573c     MSVCRT:dll_dllmain.obj
 0002:0000074c       ??_7exception@std@@6B@     1000574c     MSVCRT:throw_bad_alloc.obj
 0002:00000754       ??_C@_0BC@EOODALEL@Unknown?5exception@ 10005754     MSVCRT:throw_bad_alloc.obj
 0002:0000076c       ??_7bad_alloc@std@@6B@     1000576c     MSVCRT:throw_bad_alloc.obj
 0002:00000774       ??_C@_0P@GHFPNOJB@bad?5allocation@ 10005774     MSVCRT:throw_bad_alloc.obj
 0002:00000788       ??_7bad_array_new_length@std@@6B@ 10005788     MSVCRT:throw_bad_alloc.obj
 0002:00000790       ??_C@_0BF@KINCDENJ@bad?5array?5new?5length@ 10005790     MSVCRT:throw_bad_alloc.obj
 0002:000007ac       ??_7type_info@@6B@         100057ac     MSVCRT:std_type_info_static.obj
 0002:000007b0       __load_config_used         100057b0     MSVCRT:loadcfg.obj
 0002:00000900       ??_R4exception@std@@6B@    10005900     MSVCRT:throw_bad_alloc.obj
 0002:00000914       ??_R3exception@std@@8      10005914     MSVCRT:throw_bad_alloc.obj
 0002:00000924       ??_R2exception@std@@8      10005924     MSVCRT:throw_bad_alloc.obj
 0002:0000092c       ??_R1A@?0A@EA@exception@std@@8 1000592c     MSVCRT:throw_bad_alloc.obj
 0002:00000948       ??_R4bad_alloc@std@@6B@    10005948     MSVCRT:throw_bad_alloc.obj
 0002:0000095c       ??_R3bad_alloc@std@@8      1000595c     MSVCRT:throw_bad_alloc.obj
 0002:0000096c       ??_R2bad_alloc@std@@8      1000596c     MSVCRT:throw_bad_alloc.obj
 0002:00000978       ??_R1A@?0A@EA@bad_alloc@std@@8 10005978     MSVCRT:throw_bad_alloc.obj
 0002:00000994       ??_R4bad_array_new_length@std@@6B@ 10005994     MSVCRT:throw_bad_alloc.obj
 0002:000009a8       ??_R3bad_array_new_length@std@@8 100059a8     MSVCRT:throw_bad_alloc.obj
 0002:000009b8       ??_R2bad_array_new_length@std@@8 100059b8     MSVCRT:throw_bad_alloc.obj
 0002:000009c8       ??_R1A@?0A@EA@bad_array_new_length@std@@8 100059c8     MSVCRT:throw_bad_alloc.obj
 0002:000009e4       ??_R4type_info@@6B@        100059e4     MSVCRT:std_type_info_static.obj
 0002:000009f8       ??_R3type_info@@8          100059f8     MSVCRT:std_type_info_static.obj
 0002:00000a08       ??_R2type_info@@8          10005a08     MSVCRT:std_type_info_static.obj
 0002:00000a10       ??_R1A@?0A@EA@type_info@@8 10005a10     MSVCRT:std_type_info_static.obj
 0002:00000a2c       ___safe_se_handler_table   10005a2c     <linker-defined>
 0002:00000a34       ___volatile_metadata       10005a34     <linker-defined>
 0002:00000df8       ___rtc_iaa                 10005df8     MSVCRT:initsect.obj
 0002:00000dfc       ___rtc_izz                 10005dfc     MSVCRT:initsect.obj
 0002:00000e00       ___rtc_taa                 10005e00     MSVCRT:initsect.obj
 0002:00000e04       ___rtc_tzz                 10005e04     MSVCRT:initsect.obj
 0002:00001144       __TI2?AVbad_alloc@std@@    10006144     MSVCRT:throw_bad_alloc.obj
 0002:00001154       __CTA2?AVbad_alloc@std@@   10006154     MSVCRT:throw_bad_alloc.obj
 0002:00001160       __CT??_R0?AVbad_alloc@std@@@8??0bad_alloc@std@@QAE@ABV01@@Z12 10006160     MSVCRT:throw_bad_alloc.obj
 0002:0000117c       __CT??_R0?AVexception@std@@@8??0exception@std@@QAE@ABV01@@Z12 1000617c     MSVCRT:throw_bad_alloc.obj
 0002:00001198       __TI3?AVbad_array_new_length@std@@ 10006198     MSVCRT:throw_bad_alloc.obj
 0002:000011a8       __CTA3?AVbad_array_new_length@std@@ 100061a8     MSVCRT:throw_bad_alloc.obj
 0002:000011b8       __CT??_R0?AVbad_array_new_length@std@@@8??0bad_array_new_length@std@@QAE@ABV01@@Z12 100061b8     MSVCRT:throw_bad_alloc.obj
 0002:000017ec       __IMPORT_DESCRIPTOR_CRYPT32 100067ec     Crypt32:CRYPT32.dll
 0002:00001800       __IMPORT_DESCRIPTOR_ADVAPI32 10006800     advapi32:ADVAPI32.dll
 0002:00001814       __IMPORT_DESCRIPTOR_ncrypt 10006814     ncrypt:ncrypt.dll
 0002:00001828       __IMPORT_DESCRIPTOR_KERNEL32 10006828     kernel32:KERNEL32.dll
 0002:0000183c       __IMPORT_DESCRIPTOR_VCRUNTIME140 1000683c     vcruntime:VCRUNTIME140.dll
 0002:00001850       __IMPORT_DESCRIPTOR_api-ms-win-crt-stdio-l1-1-0 10006850     ucrt:api-ms-win-crt-stdio-l1-1-0.dll
 0002:00001864       __IMPORT_DESCRIPTOR_api-ms-win-crt-convert-l1-1-0 10006864     ucrt:api-ms-win-crt-convert-l1-1-0.dll
 0002:00001878       __IMPORT_DESCRIPTOR_api-ms-win-crt-environment-l1-1-0 10006878     ucrt:api-ms-win-crt-environment-l1-1-0.dll
 0002:0000188c       __IMPORT_DESCRIPTOR_api-ms-win-crt-string-l1-1-0 1000688c     ucrt:api-ms-win-crt-string-l1-1-0.dll
 0002:000018a0       __IMPORT_DESCRIPTOR_api-ms-win-crt-runtime-l1-1-0 100068a0     ucrt:api-ms-win-crt-runtime-l1-1-0.dll
 0002:000018b4       __IMPORT_DESCRIPTOR_api-ms-win-crt-heap-l1-1-0 100068b4     ucrt:api-ms-win-crt-heap-l1-1-0.dll
 0002:000018c8       __NULL_IMPORT_DESCRIPTOR   100068c8     Crypt32:CRYPT32.dll
 0003:00000000       ___security_cookie_complement 10008000     MSVCRT:gs_cookie.obj
 0003:00000004       ___security_cookie         10008004     MSVCRT:gs_cookie.obj
 0003:00000008       ___scrt_native_dllmain_reason 10008008     MSVCRT:utility.obj
 0003:0000000c       ___isa_enabled             1000800c     MSVCRT:cpu_disp.obj
 0003:00000010       ___scrt_ucrt_dll_is_in_use 10008010     MSVCRT:ucrt_stubs.obj
 0003:00000014       ??_R0?AVbad_alloc@std@@@8  10008014     MSVCRT:throw_bad_alloc.obj
 0003:00000030       ??_R0?AVexception@std@@@8  10008030     MSVCRT:throw_bad_alloc.obj
 0003:0000004c       ??_R0?AVbad_array_new_length@std@@@8 1000804c     MSVCRT:throw_bad_alloc.obj
 0003:00000074       ??_R0?AVtype_info@@@8      10008074     MSVCRT:std_type_info_static.obj
 0003:00000090       ?_OptionsStorage@?1??__local_stdio_printf_options@@9@4_KA 10008090     security.obj
 0003:00000098       _trace                     10008098     security.obj
 0003:000003c0       ?__type_info_root_node@@3U__type_info_node@@A 100083c0     MSVCRT:tncleanup.obj
 0003:000003c8       ?_OptionsStorage@?1??__local_stdio_scanf_options@@9@4_KA 100083c8     MSVCRT:default_local_stdio_options.obj
 0003:000003d0       ___scrt_current_native_startup_state 100083d0     MSVCRT:utility.obj
 0003:000003d4       ___scrt_native_startup_lock 100083d4     MSVCRT:utility.obj
 0003:000003f4       ___scrt_debugger_hook_flag 100083f4     MSVCRT:utility_desktop.obj
 0003:000003f8       ___isa_available           100083f8     MSVCRT:cpu_disp.obj
 0003:000003fc       ___favor                   100083fc     MSVCRT:cpu_disp.obj
 0003:00000400       ___dyn_tls_init_callback   10008400     <common>

 entry point at        0001:00002f4f

 Static symbols

 0000:ffff5000       .debug$S                   10000000     sunmscapi.exp
 0000:ffff5000       .debug$S                   10000000     vcruntime:VCRUNTIME140.dll
 0000:ffff5000       .debug$S                   10000000     vcruntime:VCRUNTIME140.dll
 0000:ffff5000       .debug$S                   10000000     vcruntime:VCRUNTIME140.dll
 0000:ffff5000       .debug$S                   10000000     vcruntime:VCRUNTIME140.dll
 0000:ffff5000       .debug$S                   10000000     vcruntime:VCRUNTIME140.dll
 0000:ffff5000       .debug$S                   10000000     vcruntime:VCRUNTIME140.dll
 0000:ffff5000       .debug$S                   10000000     vcruntime:VCRUNTIME140.dll
 0000:ffff5000       .debug$S                   10000000     vcruntime:VCRUNTIME140.dll
 0000:ffff5000       .debug$S                   10000000     vcruntime:VCRUNTIME140.dll
 0000:ffff5000       .debug$S                   10000000     vcruntime:VCRUNTIME140.dll
 0000:ffff5000       .debug$S                   10000000     ucrt:api-ms-win-crt-convert-l1-1-0.dll
 0000:ffff5000       .debug$S                   10000000     ucrt:api-ms-win-crt-environment-l1-1-0.dll
 0000:ffff5000       .debug$S                   10000000     ucrt:api-ms-win-crt-heap-l1-1-0.dll
 0000:ffff5000       .debug$S                   10000000     ucrt:api-ms-win-crt-heap-l1-1-0.dll
 0000:ffff5000       .debug$S                   10000000     ucrt:api-ms-win-crt-heap-l1-1-0.dll
 0000:ffff5000       .debug$S                   10000000     ucrt:api-ms-win-crt-runtime-l1-1-0.dll
 0000:ffff5000       .debug$S                   10000000     ucrt:api-ms-win-crt-runtime-l1-1-0.dll
 0000:ffff5000       .debug$S                   10000000     ucrt:api-ms-win-crt-runtime-l1-1-0.dll
 0000:ffff5000       .debug$S                   10000000     ucrt:api-ms-win-crt-runtime-l1-1-0.dll
 0000:ffff5000       .debug$S                   10000000     ucrt:api-ms-win-crt-runtime-l1-1-0.dll
 0000:ffff5000       .debug$S                   10000000     ucrt:api-ms-win-crt-runtime-l1-1-0.dll
 0000:ffff5000       .debug$S                   10000000     ucrt:api-ms-win-crt-runtime-l1-1-0.dll
 0000:ffff5000       .debug$S                   10000000     ucrt:api-ms-win-crt-runtime-l1-1-0.dll
 0000:ffff5000       .debug$S                   10000000     ucrt:api-ms-win-crt-runtime-l1-1-0.dll
 0000:ffff5000       .debug$S                   10000000     ucrt:api-ms-win-crt-runtime-l1-1-0.dll
 0000:ffff5000       .debug$S                   10000000     ucrt:api-ms-win-crt-runtime-l1-1-0.dll
 0000:ffff5000       .debug$S                   10000000     ucrt:api-ms-win-crt-runtime-l1-1-0.dll
 0000:ffff5000       .debug$S                   10000000     ucrt:api-ms-win-crt-stdio-l1-1-0.dll
 0000:ffff5000       .debug$S                   10000000     ucrt:api-ms-win-crt-stdio-l1-1-0.dll
 0000:ffff5000       .debug$S                   10000000     ucrt:api-ms-win-crt-stdio-l1-1-0.dll
 0000:ffff5000       .debug$S                   10000000     ucrt:api-ms-win-crt-stdio-l1-1-0.dll
 0000:ffff5000       .debug$S                   10000000     ucrt:api-ms-win-crt-string-l1-1-0.dll
 0000:ffff5000       .debug$S                   10000000     ucrt:api-ms-win-crt-string-l1-1-0.dll
 0000:ffff5000       .debug$S                   10000000     Crypt32:CRYPT32.dll
 0000:ffff5000       .debug$S                   10000000     Crypt32:CRYPT32.dll
 0000:ffff5000       .debug$S                   10000000     Crypt32:CRYPT32.dll
 0000:ffff5000       .debug$S                   10000000     Crypt32:CRYPT32.dll
 0000:ffff5000       .debug$S                   10000000     Crypt32:CRYPT32.dll
 0000:ffff5000       .debug$S                   10000000     Crypt32:CRYPT32.dll
 0000:ffff5000       .debug$S                   10000000     Crypt32:CRYPT32.dll
 0000:ffff5000       .debug$S                   10000000     Crypt32:CRYPT32.dll
 0000:ffff5000       .debug$S                   10000000     Crypt32:CRYPT32.dll
 0000:ffff5000       .debug$S                   10000000     Crypt32:CRYPT32.dll
 0000:ffff5000       .debug$S                   10000000     Crypt32:CRYPT32.dll
 0000:ffff5000       .debug$S                   10000000     Crypt32:CRYPT32.dll
 0000:ffff5000       .debug$S                   10000000     Crypt32:CRYPT32.dll
 0000:ffff5000       .debug$S                   10000000     Crypt32:CRYPT32.dll
 0000:ffff5000       .debug$S                   10000000     advapi32:ADVAPI32.dll
 0000:ffff5000       .debug$S                   10000000     advapi32:ADVAPI32.dll
 0000:ffff5000       .debug$S                   10000000     advapi32:ADVAPI32.dll
 0000:ffff5000       .debug$S                   10000000     advapi32:ADVAPI32.dll
 0000:ffff5000       .debug$S                   10000000     advapi32:ADVAPI32.dll
 0000:ffff5000       .debug$S                   10000000     advapi32:ADVAPI32.dll
 0000:ffff5000       .debug$S                   10000000     advapi32:ADVAPI32.dll
 0000:ffff5000       .debug$S                   10000000     advapi32:ADVAPI32.dll
 0000:ffff5000       .debug$S                   10000000     advapi32:ADVAPI32.dll
 0000:ffff5000       .debug$S                   10000000     advapi32:ADVAPI32.dll
 0000:ffff5000       .debug$S                   10000000     advapi32:ADVAPI32.dll
 0000:ffff5000       .debug$S                   10000000     advapi32:ADVAPI32.dll
 0000:ffff5000       .debug$S                   10000000     advapi32:ADVAPI32.dll
 0000:ffff5000       .debug$S                   10000000     advapi32:ADVAPI32.dll
 0000:ffff5000       .debug$S                   10000000     advapi32:ADVAPI32.dll
 0000:ffff5000       .debug$S                   10000000     advapi32:ADVAPI32.dll
 0000:ffff5000       .debug$S                   10000000     advapi32:ADVAPI32.dll
 0000:ffff5000       .debug$S                   10000000     advapi32:ADVAPI32.dll
 0000:ffff5000       .debug$S                   10000000     kernel32:KERNEL32.dll
 0000:ffff5000       .debug$S                   10000000     kernel32:KERNEL32.dll
 0000:ffff5000       .debug$S                   10000000     kernel32:KERNEL32.dll
 0000:ffff5000       .debug$S                   10000000     kernel32:KERNEL32.dll
 0000:ffff5000       .debug$S                   10000000     kernel32:KERNEL32.dll
 0000:ffff5000       .debug$S                   10000000     kernel32:KERNEL32.dll
 0000:ffff5000       .debug$S                   10000000     kernel32:KERNEL32.dll
 0000:ffff5000       .debug$S                   10000000     kernel32:KERNEL32.dll
 0000:ffff5000       .debug$S                   10000000     kernel32:KERNEL32.dll
 0000:ffff5000       .debug$S                   10000000     kernel32:KERNEL32.dll
 0000:ffff5000       .debug$S                   10000000     kernel32:KERNEL32.dll
 0000:ffff5000       .debug$S                   10000000     kernel32:KERNEL32.dll
 0000:ffff5000       .debug$S                   10000000     kernel32:KERNEL32.dll
 0000:ffff5000       .debug$S                   10000000     kernel32:KERNEL32.dll
 0000:ffff5000       .debug$S                   10000000     kernel32:KERNEL32.dll
 0000:ffff5000       .debug$S                   10000000     kernel32:KERNEL32.dll
 0000:ffff5000       .debug$S                   10000000     ncrypt:ncrypt.dll
 0000:ffff5000       .debug$S                   10000000     ncrypt:ncrypt.dll
 0000:ffff5000       .debug$S                   10000000     ncrypt:ncrypt.dll
 0000:ffff5000       .debug$S                   10000000     ncrypt:ncrypt.dll
 0000:ffff5000       .debug$S                   10000000     ncrypt:ncrypt.dll
 0000:ffff5000       .debug$S                   10000000     ncrypt:ncrypt.dll
 0000:ffff5000       .debug$S                   10000000     ncrypt:ncrypt.dll
 0000:ffff5000       .debug$S                   10000000     ncrypt:ncrypt.dll
 0001:00000000       ??__Etrace@@YAXXZ          10001000 f   security.obj
 0001:00002b40       $$000000                   10003b40     MSVCRT:sehprolg4.obj
 0001:00002b90       $$000000                   10003b90     MSVCRT:sehprolg4gs.obj
 0001:00002c0f       ?dllmain_crt_dispatch@@YGHQAUHINSTANCE__@@KQAX@Z 10003c0f f   MSVCRT:dll_dllmain.obj
 0001:00002c62       ?dllmain_crt_process_attach@@YAHQAUHINSTANCE__@@QAX@Z 10003c62 f   MSVCRT:dll_dllmain.obj
 0001:00002d69       ?dllmain_crt_process_detach@@YAH_N@Z 10003d69 f   MSVCRT:dll_dllmain.obj
 0001:00002e19       ?dllmain_dispatch@@YAHQAUHINSTANCE__@@KQAX@Z 10003e19 f   MSVCRT:dll_dllmain.obj
 0001:00002f24       ?dllmain_raw@@YGHQAUHINSTANCE__@@KQAX@Z 10003f24 f   MSVCRT:dll_dllmain.obj
 0001:00002faf       __catch$??2@YAPAXIABUnothrow_t@std@@@Z$0 10003faf f   MSVCRT:new_scalar_nothrow.obj
 0001:000030ee       ___get_entropy             100040ee f   MSVCRT:gs_support.obj
 0001:000031e3       ?find_pe_section@@YAPAU_IMAGE_SECTION_HEADER@@QAEI@Z 100041e3 f   MSVCRT:utility.obj
 0001:00003a97       __ehhandler$??2@YAPAXIABUnothrow_t@std@@@Z 10004a97 f   MSVCRT:new_scalar_nothrow.obj
 0002:0000017c       ?trace$initializer$@@3P6AXXZA 1000517c     security.obj
 0002:00000740       _GS_ExceptionPointers      10005740     MSVCRT:gs_report.obj
 0002:00000e08       __sehtable$_Java_sun_security_mscapi_CKeyStore_loadKeysOrCertificateChains@12 10005e08     security.obj
 0002:00000e28       __sehtable$_Java_sun_security_mscapi_CKeyStore_storeCertificate@40 10005e28     security.obj
 0002:00000e48       __sehtable$_Java_sun_security_mscapi_CKeyStore_removeCertificate@24 10005e48     security.obj
 0002:00000e68       __sehtable$_Java_sun_security_mscapi_CKeyStore_destroyKeyContainer@12 10005e68     security.obj
 0002:00000e88       __sehtable$_Java_sun_security_mscapi_CKeyStore_storePrivateKey@24 10005e88     security.obj
 0002:00000ea8       __sehtable$_Java_sun_security_mscapi_CRSACipher_encryptDecrypt@32 10005ea8     security.obj
 0002:00000ec8       __sehtable$_Java_sun_security_mscapi_CKeyPairGenerator_00024RSA_generateCKeyPair@20 10005ec8     security.obj
 0002:00000ee8       __sehtable$_Java_sun_security_mscapi_CPublicKey_getPublicKeyBlob@24 10005ee8     security.obj
 0002:00000f08       __sehtable$_Java_sun_security_mscapi_CPublicKey_00024CRSAPublicKey_getExponent@12 10005f08     security.obj
 0002:00000f28       __sehtable$_Java_sun_security_mscapi_CPublicKey_00024CRSAPublicKey_getModulus@12 10005f28     security.obj
 0002:00000f48       __sehtable$_Java_sun_security_mscapi_CSignature_signCngHash@44 10005f48     security.obj
 0002:00000f68       __sehtable$_Java_sun_security_mscapi_CSignature_verifyCngSignedHash@52 10005f68     security.obj
 0002:00000f88       __sehtable$_Java_sun_security_mscapi_CSignature_signHash@40 10005f88     security.obj
 0002:00000fa8       __sehtable$_Java_sun_security_mscapi_CSignature_verifySignedHash@44 10005fa8     security.obj
 0002:00000fc8       __sehtable$_Java_sun_security_mscapi_CSignature_importPublicKey@20 10005fc8     security.obj
 0002:00000fe8       __sehtable$_Java_sun_security_mscapi_CSignature_importECPublicKey@20 10005fe8     security.obj
 0002:00001008       __sehtable$_Java_sun_security_mscapi_PRNG_generateSeed@16 10006008     security.obj
 0002:00001028       __sehtable$_convertToLittleEndian 10006028     security.obj
 0002:00001048       __sehtable$_generateKeyBlob 10006048     security.obj
 0002:00001068       __sehtable$?dllmain_crt_process_attach@@YAHQAUHINSTANCE__@@QAX@Z 10006068     MSVCRT:dll_dllmain.obj
 0002:00001088       __sehtable$?dllmain_crt_process_detach@@YAH_N@Z 10006088     MSVCRT:dll_dllmain.obj
 0002:000010b0       __sehtable$?dllmain_dispatch@@YAHQAUHINSTANCE__@@KQAX@Z 100060b0     MSVCRT:dll_dllmain.obj
 0002:000010cc       __catchsym$??2@YAPAXIABUnothrow_t@std@@@Z$2 100060cc     MSVCRT:new_scalar_nothrow.obj
 0002:000010dc       __unwindtable$??2@YAPAXIABUnothrow_t@std@@@Z 100060dc     MSVCRT:new_scalar_nothrow.obj
 0002:000010ec       __tryblocktable$??2@YAPAXIABUnothrow_t@std@@@Z 100060ec     MSVCRT:new_scalar_nothrow.obj
 0002:00001100       __ehfuncinfo$??2@YAPAXIABUnothrow_t@std@@@Z 10006100     MSVCRT:new_scalar_nothrow.obj
 0002:00001128       __sehtable$___scrt_is_nonwritable_in_current_image 10006128     MSVCRT:utility.obj
 0002:000011e0       .edata                     100061e0     sunmscapi.exp
 0002:00001208       rgpv                       10006208     sunmscapi.exp
 0002:00001260       rgszName                   10006260     sunmscapi.exp
 0002:000012b8       rgwOrd                     100062b8     sunmscapi.exp
 0002:000012e4       szName                     100062e4     sunmscapi.exp
 0002:000012f2       $N00001                    100062f2     sunmscapi.exp
 0002:0000133b       $N00002                    1000633b     sunmscapi.exp
 0002:00001376       $N00003                    10006376     sunmscapi.exp
 0002:000013b7       $N00004                    100063b7     sunmscapi.exp
 0002:000013fa       $N00005                    100063fa     sunmscapi.exp
 0002:00001433       $N00006                    10006433     sunmscapi.exp
 0002:0000146b       $N00007                    1000646b     sunmscapi.exp
 0002:000014a2       $N00008                    100064a2     sunmscapi.exp
 0002:000014cc       $N00009                    100064cc     sunmscapi.exp
 0002:000014ff       $N00010                    100064ff     sunmscapi.exp
 0002:0000152c       $N00011                    1000652c     sunmscapi.exp
 0002:00001573       $N00012                    10006573     sunmscapi.exp
 0002:000015b9       $N00013                    100065b9     sunmscapi.exp
 0002:000015f2       $N00014                    100065f2     sunmscapi.exp
 0002:00001629       $N00015                    10006629     sunmscapi.exp
 0002:00001670       $N00016                    10006670     sunmscapi.exp
 0002:000016aa       $N00017                    100066aa     sunmscapi.exp
 0002:000016e2       $N00018                    100066e2     sunmscapi.exp
 0002:00001716       $N00019                    10006716     sunmscapi.exp
 0002:00001747       $N00020                    10006747     sunmscapi.exp
 0002:00001783       $N00021                    10006783     sunmscapi.exp
 0002:000017bc       $N00022                    100067bc     sunmscapi.exp
 0002:00001be4       .idata$6                   10006be4     Crypt32:CRYPT32.dll
 0002:00001d46       .idata$6                   10006d46     advapi32:ADVAPI32.dll
 0002:00001dfe       .idata$6                   10006dfe     ncrypt:ncrypt.dll
 0002:00001f50       .idata$6                   10006f50     kernel32:KERNEL32.dll
 0002:0000200a       .idata$6                   1000700a     vcruntime:VCRUNTIME140.dll
 0002:0000215a       .idata$6                   1000715a     ucrt:api-ms-win-crt-stdio-l1-1-0.dll
 0002:0000217a       .idata$6                   1000717a     ucrt:api-ms-win-crt-convert-l1-1-0.dll
 0002:0000219c       .idata$6                   1000719c     ucrt:api-ms-win-crt-environment-l1-1-0.dll
 0002:000021c2       .idata$6                   100071c2     ucrt:api-ms-win-crt-string-l1-1-0.dll
 0002:000021e4       .idata$6                   100071e4     ucrt:api-ms-win-crt-runtime-l1-1-0.dll
 0002:00002206       .idata$6                   10007206     ucrt:api-ms-win-crt-heap-l1-1-0.dll
 0003:0000009c       ?__proc_attached@@3HA      1000809c     MSVCRT:dll_dllmain.obj
 0003:000000a0       _GS_ExceptionRecord        100080a0     MSVCRT:gs_report.obj
 0003:000000f0       _GS_ContextRecord          100080f0     MSVCRT:gs_report.obj
 0003:000003d8       ?is_initialized_as_dll@@3_NA 100083d8     MSVCRT:utility.obj
 0003:000003d9       ?module_local_atexit_table_initialized@@3_NA 100083d9     MSVCRT:utility.obj
 0003:000003dc       ?module_local_atexit_table@@3U_onexit_table_t@@A 100083dc     MSVCRT:utility.obj
 0003:000003e8       ?module_local_at_quick_exit_table@@3U_onexit_table_t@@A 100083e8     MSVCRT:utility.obj
 0004:00000060       $R000000                   10009060     sunmscapi.dll.res
